:100000000C9438010C9455010C9455010C94550135
:100010000C9455010C9455010C9455010C94550108
:100020000C9455010C9455010C9455010C945501F8
:100030000C9440120C9455010C9455010C945501EC
:100040000C9455010C949C050C943F180C9455117C
:100050000C94DF110C9455010C9455010C9455012E
:100060000C9455010C9455010C9455010C945501B8
:100070004570692D4F5344205665722E302E392E0F
:10008000312E302E610000416B7475656C6C6573A8
:100090002053657474696E67000053657474696EEB
:1000A0006720200000486F6568656E73656E736F2A
:1000B000722000004853206D697420536368616C9E
:1000C00074657220000048656164696E6720486F3E
:1000D0006C642000004B6F6D706173732000004BE7
:1000E0006F6D70617373206669782000004750530C
:1000F00020416B74697620000041636873656E6B04
:100100006F7070656C756E67200000447265687270
:1001100061746520626567722E2000004665686C18
:1001200065722046433C2D3E4F5344200000556EDF
:100130007465727370616E6E756E672000004B653A
:10014000696E652053657474696E672D416E7A65BA
:10015000696765000050432F425420616B746976D3
:10016000000055656265726E65686D65204C65744A
:100170007A7465732053657474696E6700004B650B
:10018000696E65204465766976652D416E7A65698C
:100190006765000050432F425420616B74697600FC
:1001A0000055656265726E65686D65204C65747A90
:1001B0007465732044657669636500004F4E0000E6
:1001C0002D2D2D000044657669636520756E6420D1
:1001D00056657273696F6E736162667261676500FE
:1001E0000044656369766520202020203D200000C2
:1001F00046572D56657273696F6E203D200000468C
:100200004300004E43000046432D6F6C6420465768
:1002100000004550492D4D656E750050616C0050D1
:10022000432F4254004B656E6E756E670052432D2E
:1002300042657472696562004550492D5374726F4E
:100240006D0045786974004F4E002D2D0076767D47
:1002500076767A76767E76767776767B767678762A
:10026000767C76767976767D76767A76767E760088
:1002700011241FBECFEFD4E0DEBFCDBF11E0A0E060
:10028000B1E0ECE3F2E302C005900D92AA38B107A9
:10029000D9F713E0AAE8B1E001C01D92AA3AB1076C
:1002A000E1F70E9462010C941C190C94000082E991
:1002B00081BB8FE084BBAC9AAD9A8EE28ABBD99A9F
:1002C000DD9A08951092D2011092CE011092D301BE
:1002D000E199FECF80E090E09FBB8EBBE09A8DB3AA
:1002E00080939101E199FECF81E090E09FBB8EBBAE
:1002F000E09A8DB380930001E199FECF82E090E017
:100300009FBB8EBBE09A8DB380939201E199FECFA3
:1003100087E190E09FBB8EBBE09A8DB380939F01F5
:10032000E199FECF88E190E09FBB8EBBE09A8DB350
:100330008093B801E199FECF8AE190E09FBB8EBB2C
:10034000E09A8DB380930901E199FECF89E190E0B5
:100350009FBB8EBBE09A8DB38093B401E199FECF31
:100360008BE190E09FBB8EBBE09A8DB380939301AD
:1003700020910001213079F49EE09093030187E001
:100380008093040186E880930501209306019093F1
:1003900007018CE00EC09CE09093030185E0809300
:1003A00004018AE4809305011092060190930701ED
:1003B0008AE0809308010E944E1682E981BB8FE09B
:1003C00084BBAC9AAD9A8EE28ABBD99ADD9A0E9420
:1003D000950580919101813019F40E94501002C05E
:1003E0000E9440107894A89A0E94CB040E94FE05B7
:1003F0000E94F10980919301882311F00E94340A30
:100400008091BD01882311F00E9479130E94340A63
:100410000E9421118091B001813021F41092B0012D
:100420000E94EE1680918C018130E9F410928C01CB
:100430008091D201882389F48091B401843069F4D9
:1004400080919101882349F480919401813029F4AD
:1004500080E363E64AE00E94CF100E9433120E94BC
:1004600038120E94911380918F018130E1F48091C4
:10047000D2018823C1F4AA9A0E94890E0E945109D0
:100480000E9466088091BB01882321F00E94AC1273
:100490000E94B20A8091BC01882311F00E949E162E
:1004A0000E94890AAA9880918A018130A9F58091D9
:1004B000D201882389F510928A0180919F018823B7
:1004C00021F080910201833014F00E94630A809130
:1004D0009C0190919D01019690939D0180939C01B8
:1004E0000197CB9769F480919A0190919B010196B5
:1004F00090939B0180939A0110929D0110929C0110
:100500000E943D0C0E94870D80919301813021F45F
:100510000E94FC050E94FD0580918B01813009F04D
:1005200079CF8091D201882309F074CF10928B018A
:100530000E94FA098091BD01882309F46BCF0E94C3
:100540000E1368CF782FD99827E030E041E050E0D3
:10055000DB980000000000000000CA01022E02C06B
:10056000880F991F0A94E2F7872311F0DA9A01C0E5
:10057000DA980000000000000000DB9A0000000094
:1005800000000000215030408FEF2F3F380701F767
:1005900027E030E041E050E0DB9800000000000080
:1005A0000000CA01022E02C0880F991F0A94E2F7C8
:1005B000862311F0DA9A01C0DA98000000000000EA
:1005C0000000DB9A000000000000000021503040D5
:1005D0008FEF2F3F380701F7DB98DA98D99A089503
:1005E00084E064E00E94A20280E06CE40E94A20227
:1005F00010928C0180918C018823E1F38CE66AE0F3
:100600000E94A20285E060E00E94A20208951F936A
:100610008091B401823051F40E94601010928A01DE
:1006200080918A018823E1F310928A0182E661E7D2
:100630004FEF0E94CF1010928A0110E00DC0809100
:100640008F01813011F40E94890E80918A018130DE
:1006500019F410928A0111E08091BA01882311F4F3
:10066000112369F38091B401823011F40E94A71024
:10067000112309F0D9C080919A03809309018091D8
:100680008A038093B8012091B801E199FECF88E1F7
:1006900090E09FBB8EBB2DBB0FB6F894E29AE19A17
:1006A0000FBE20910901E199FECF8AE190E09FBB46
:1006B0008EBB2DBB0FB6F894E29AE19A0FBE82E092
:1006C00061E047E850E00E94C40D82E062E04AE940
:1006D00050E00E94C40D82E064E045EA50E00E94D0
:1006E000C40D82E065E044EB50E00E94C40D82E05E
:1006F00066E046EC50E00E94C40D82E067E045ED04
:1007000050E00E94C40D82E068E04FED50E00E948E
:10071000C40D82E069E04DEE50E00E94C40D82E01D
:100720006AE049EF50E00E94C40D82E06BE04EE2C7
:1007300051E00E94C40D4091B6015091B70184E18F
:1007400062E00E94990D8091B80180FF05C084E1AC
:1007500064E04CEB51E004C084E164E040EC51E023
:100760000E94C40D8091B80181FF05C084E165E05D
:100770004CEB51E004C084E165E040EC51E00E94A4
:10078000C40D8091B80182FF05C084E166E04CEBA6
:1007900051E004C084E166E040EC51E00E94C40DE9
:1007A0008091B80183FF05C084E167E04CEB51E024
:1007B00004C084E167E040EC51E00E94C40D8091E8
:1007C000B80184FF05C084E168E04CEB51E004C04F
:1007D00084E168E040EC51E00E94C40D8091B801D2
:1007E00085FF05C084E169E04CEB51E004C084E181
:1007F00069E040EC51E00E94C40D8091B80186FF91
:1008000005C084E16AE04CEB51E004C084E16AE099
:1008100040EC51E00E94C40D40919A0384E16BE0EA
:1008200050E00E94990D20C082E062E047E850E06D
:100830000E94C40D82E065E04CE151E00E94C40DCD
:10084000E199FECF88E190E09FBB8EBBE09A8DB32B
:1008500080938A03E199FECF8AE190E09FBB8EBB33
:10086000E09A8DB38093090190918A03892F81705A
:100870008093BB01892F88708093BC01892F80727F
:100880008093BD0194709093BE011F9108951F93B2
:1008900080918A018823E1F310928A0183E666E75A
:1008A00040E00E94CF1010E00DC080918F01813098
:1008B00011F40E946C0E80918A01813019F410921B
:1008C0008A0111E08091B501882311F4112369F3A5
:1008D000112309F054C082E062E045EC51E00E942F
:1008E000C40D82E064E041EE51E00E94C40D82E05C
:1008F00066E040EF51E00E94C40D8091B401813068
:1009000031F48EE064E04FEF51E00E94C40D80911D
:10091000B401823031F48EE064E043E052E00E94A2
:10092000C40D8091B401843031F48EE064E047E07E
:1009300052E00E94C40D409144038EE066E050E016
:100940000E94990D4091450380E166E050E00E94CD
:10095000990D4091460383E166E050E00E94990DB5
:100960002091B401E199FECF89E190E09FBB8EBB5D
:100970002DBB0FB6F894E29AE19A0FBE0AC0E19936
:10098000FECF89E190E09FBB8EBBE09A8DB3809350
:10099000B4011F9108950E94F00283E66FE644E6D9
:1009A0000E94CF1010928A0180918A018823E1F37E
:1009B00087E062E040E750E00E94C40D0E94FF051E
:1009C00010928A0180918A018823E1F310928A01B2
:1009D00080918A018823E1F310928A0180918A0133
:1009E0008823E1F310928A0184E064E00E94A2026D
:1009F00080E06CE40E94A20280919101882319F4A6
:100A00000E9447041CC082E062E04EE751E00E9471
:100A1000C40D82E064E044E951E00E94C40D82E02C
:100A200066E041EA51E00E94C40DE199FECF89E100
:100A300090E09FBB8EBBE09A8DB38093B401809110
:100A40008A018823E1F310928A0180918A01882328
:100A5000E1F310928A0184E064E00E94A20280E047
:100A60006CE40E94A20280919101882319F40E94F3
:100A7000070326C082E062E04EE351E00E94C40D0D
:100A800082E064E045E551E00E94C40D82E066E04A
:100A900042E651E00E94C40DE199FECF88E190E06A
:100AA0009FBB8EBBE09A8DB38093B801E199FECFD6
:100AB0008AE190E09FBB8EBBE09A8DB380930901E1
:100AC0008091B401823029F483E66FE64AE00E9407
:100AD000CF108091B401813029F482E664E64AE0C7
:100AE0000E94CF1080918A018823E1F310928A013D
:100AF00080918A018823E1F310928A0180918A0112
:100B00008823E1F310928A0180918A018823E1F31E
:100B100010928A0180918A018823E1F310928A0160
:100B200084E064E00E94A202089582E083BF82E430
:100B30008EBD8AE089BF08951F920F920FB60F9263
:100B400011248F939F9380918E018F5F80938E01EC
:100B500080918E01883449F591E090938D01109237
:100B60008E0180919E038F5F80939E0380919E03F0
:100B7000843631F410929E0390938A0190938B01F6
:100B800080919E03823319F481E080938B018091E0
:100B90009D038F5F80939D0380919D038A3029F48C
:100BA00010929D0381E080938C019F918F910F9013
:100BB0000FBE0F901F901895982F80538A3010F019
:100BC00020E005C0903311F42AE001C0282F892FBE
:100BD00081548A3110F4292F2653892F81568A3166
:100BE00010F4292F2C539D3211F429E403C09E32B6
:100BF00009F421E4822F089508950895089585E069
:100C000060E00E94A20286E063E80E94A20287E000
:100C100060E90E94A20285E060E00E94A20286E0F4
:100C200064E80E94A20287E061E90E94A20285E0D6
:100C300060E00E94A20286E065E80E94A20287E0CE
:100C400062E90E94A20285E060E00E94A20286E0C2
:100C500066E80E94A20287E063E90E94A20285E0A2
:100C600060E00E94A20286E067E80E94A20287E09C
:100C700064E90E94A20285E060E00E94A20286E090
:100C800068E80E94A20287E065E90E94A20285E06E
:100C900060E00E94A20286E069E80E94A20287E06A
:100CA00066E90E94A20285E060E00E94A20286E05E
:100CB0006AE80E94A20287E067E90E94A20285E03A
:100CC00060E00E94A20286E061EA0E94A20287E040
:100CD00068E90E94A20285E060E00E94A20286E02C
:100CE00062EA0E94A20287E069E90E94A20285E00E
:100CF00060E00E94A20286E063EA0E94A20287E00E
:100D00006AE90E94A20285E060E00E94A20286E0F9
:100D100064EA0E94A20287E06BE90E94A20285E0D9
:100D200060E00E94A20286E065EA0E94A20287E0DB
:100D30006CE90E94A20285E060E00E94A20286E0C7
:100D400066EA0E94A20287E06DE90E94A20285E0A5
:100D500060E00E94A20286E067EA0E94A20287E0A9
:100D60006EE90E94A20285E060E00E94A20286E095
:100D700068EA0E94A20287E06FE90E94A20285E071
:100D800060E00E94A20286E06FEB0E94A20287E070
:100D900060EA0E94A20285E060E00E94A20286E072
:100DA00060EC0E94A20287E061EA0E94A20285E054
:100DB00060E00E94A20286E061EC0E94A20287E04D
:100DC00062EA0E94A20285E060E00E94A20286E040
:100DD00062EC0E94A20287E063EA0E94A20285E020
:100DE00060E00E94A20286E063EC0E94A20287E01B
:100DF00064EA0E94A20285E060E00E94A20286E00E
:100E000064EC0E94A20287E065EA0E94A20285E0EB
:100E100060E00E94A20286E065EC0E94A20287E0E8
:100E200066EA0E94A20285E060E00E94A20286E0DB
:100E300066EC0E94A20287E067EA0E94A20285E0B7
:100E400060E00E94A20286E06DED0E94A20287E0AF
:100E500068EA0E94A20285E060E00E94A20286E0A9
:100E60006EED0E94A20287E069EA0E94A20285E07C
:100E700060E00E94A20286E06FED0E94A20287E07D
:100E80006AEA0E94A20285E060E00E94A20286E077
:100E900060EE0E94A20287E06BEA0E94A20285E057
:100EA00060E00E94A20286E061EE0E94A20287E05A
:100EB0006CEA0E94A20285E060E00E94A20286E045
:100EC00062EE0E94A20287E06DEA0E94A20285E023
:100ED00060E00E94A20286E063EE0E94A20287E028
:100EE0006EEA0E94A20285E060E00E94A20286E013
:100EF00064EE0E94A20287E06FEA0E94A20285E0EF
:100F000060E00E94A20286E06BEF0E94A20287E0EE
:100F100060EB0E94A20285E060E00E94A20286E0EF
:100F20006CEF0E94A20287E061EB0E94A20285E0C2
:100F300060E00E94A20286E06DEF0E94A20287E0BC
:100F400062EB0E94A20285E060E00E94A20286E0BD
:100F50006EEF0E94A20287E063EB0E94A20285E08E
:100F600060E00E94A20286E06FEF0E94A20287E08A
:100F700064EB0E94A20285E061E00E94A20286E08A
:100F800060E00E94A20287E065EB0E94A20285E079
:100F900061E00E94A20286E061E00E94A20287E076
:100FA00066EB0E94A2020895BF92CF92DF92EF9269
:100FB000FF920F931F93CF93DF937C01B62E8C018A
:100FC00045E0C42ED12CC80ED91E862F90E0EC012E
:100FD000CC0FDD1FC80FD91FCA5EDE4F0EC085E0E3
:100FE000612F0E94A20286E0602F0E94A20287E089
:100FF00068810E94A2020F5F1F4F0C151D0578F338
:101000008701065F1F4F8FE090E0E80EF91E8B2DE1
:1010100090E0EC01CC0FDD1FC80FD91FCA5EDE4F78
:101020000EC085E0612F0E94A20286E0602F0E9420
:10103000A20287E068810E94A2020F5F1F4F0E1577
:101040001F0578F3DF91CF911F910F91FF90EF90E3
:10105000DF90CF90BF900895EF92FF920F931F9370
:10106000CF93DF938C01EC0155E0E52EF12CE80ED7
:10107000F91E0DC085E06D2F0E94A20286E06C2F44
:101080000E94A20287E060E00E94A2022196CE1593
:10109000DF0580F3E8012A96015F1F4F0DC085E050
:1010A0006D2F0E94A20286E06C2F0E94A20287E0B0
:1010B00060E00E94A2022196C017D10780F3DF9161
:1010C000CF911F910F91FF90EF9008951F93CF93B1
:1010D000DF93C0914402D0914502D7FD12C0CE01EA
:1010E0006AE070E00E940919182F169520910401FA
:1010F00030E0CE016AE070E00E940919261B310938
:1011000018C0EE27FF27EC1BFD0BCF016AE070E053
:101110000E940919182F16951C5F2091040130E0D8
:101120002F5F3F4FCF016AE070E00E940919260F40
:10113000311DE90175E0CC0FDD1F7A95E1F7220F33
:10114000331FC21BD30B279680911201909113017C
:10115000C817D90739F080911201909113010E94AC
:101160002C0804C08091C101811721F0CE01612FAC
:101170000E94D4071093C101D0931301C0931201B0
:10118000DF91CF911F910895CF92DF92EF92FF925E
:101190000F931F93CF93DF938C01E62E85E0612F91
:1011A0000E94A20286E0602F0E94A202CE2CDD24C3
:1011B00084E391E0C80ED91E87E0F60160810E94A9
:1011C000A202EEE1EE2EF12CE00EF11E85E06F2D75
:1011D0000E94A20286E06E2D0E94A20287E0F60124
:1011E00060810E94A202E801CC54DF4F025F1E4FD3
:1011F00085E06D2F0E94A20286E06C2F0E94A20261
:1012000087E0F60160810E94A2026E96C017D107A6
:1012100079F7DF91CF911F910F91FF90EF90DF90C1
:10122000CF900895EF92FF920F931F93CF93DF9388
:101230007C0185E06F2D0E94A20286E06E2D0E9447
:10124000A20287E060E00E94A2028701025E1F4FB7
:1012500085E0612F0E94A20286E0602F0E94A20218
:1012600087E060E00E94A202E701CC54DF4F8701D3
:10127000025F1E4F85E06D2F0E94A20286E06C2F58
:101280000E94A20287E060E00E94A2026E96C01750
:10129000D10781F7DF91CF911F910F91FF90EF90D0
:1012A00008951F93CF93DF93E0914202F0914302A0
:1012B000F7FD14C0CF016AE070E00E940919182FF1
:1012C00016951C5F80910501C82FD0E0CF016AE020
:1012D00070E00E940919C61BD10917C022273327C5
:1012E0002E1B3F0BC9016AE070E00E940919182FFC
:1012F000169580910501C82FD0E02196C9016AE0BA
:1013000070E00E940919C60FD11D809114019091BF
:101310001501C817D90739F0809114019091150172
:101320000E94120904C08091C201811721F0CE01F0
:10133000612F0E94C4081093C201D0931501C0937D
:101340001401DF91CF911F91089585E060E00E9424
:10135000A20286E06FEC0E94A20287E06CE80E9485
:10136000A20285E061E00E94A20286E06BE00E949A
:10137000A20287E06DE80E94A2020895EF92FF9218
:101380000F931F93CF93DF937A019EE1699FB00182
:101390001124680F711D8B01020F111D10929F0304
:1013A000EB0115C085E06D2F0E94A20286E06C2F34
:1013B0000E94A20280919F03F701E80FF11D608156
:1013C0008F5F80939F0387E00E94A2022196C0173F
:1013D000D10740F3DF91CF911F910F91FF90EF90D4
:1013E00008956091030181E04DE051E025E00E9405
:1013F000BE090895DF93CF9300D000D0CDB7DEB7FC
:1014000019821A821C82F89430914A027894832FB0
:101410006AE00E94E918282F0E94E918482F822FBD
:101420000E94E918292F832F0E94E918992319F4A3
:101430008AE08C8301C09C83222319F48AE08A838A
:1014400001C02A83498385E48B8383E061E0AE0198
:101450004F5F5F4F24E00E94BE090F900F900F90E6
:101460000F90CF91DF910895DF93CF9300D000D0FC
:10147000CDB7DEB780E289839BE09A8381E38B83DB
:101480009C8381E061E0AE014F5F5F4F21E00E94ED
:10149000BE0980919301813079F462E0AE014E5F24
:1014A0005F4F21E00E94BE0981E063E0AE014D5F25
:1014B0005F4F22E00E94BE090F900F900F900F9097
:1014C000CF91DF910895DF93CF9300D000D00F929A
:1014D000CDB7DEB7DE011196E1E4F1E085E00190E1
:1014E0000D928150E1F7609104018CE0AE014F5FF5
:1014F0005F4F25E00E94BE090F900F900F900F9054
:101500000F90CF91DF91089580E06CE40E94A202D9
:1015100008958091180390911903843B910554F02C
:1015200080919A0390E0209116033091170382175F
:10153000930744F08091C301882371F481E0809384
:10154000C30108958091C301181624F480E06CE46F
:101550000E94A2021092C301089580E062E40E94FA
:10156000A20208958F929F92AF92BF92CF92DF9284
:10157000EF92FF920F931F93DF93CF93CDB7DEB718
:101580002F970FB6F894DEBF0FBECDBFFE013B967E
:1015900085E0DF011D928A95E9F7809146029091DE
:1015A0004702019797FF02C080E090E08E010F5F35
:1015B0001F4FB8014AE050E00E94B818F8010190AE
:1015C0000020E9F73197FE2EF01A80E0CF2CDD24C1
:1015D000C7FCD094F6E08F2E912C8C0E9D1E5801E6
:1015E0000BC0F501E00FF11F80810E94DC05080DA2
:1015F000191DF80180838E2D082F10E0E82EE3944A
:101600000C151D0574F380939F0385E169E0AE011D
:10161000455F5F4F25E00E94BE0989E18F1969E0AF
:10162000A4012F2D0E94BE092F960FB6F894DEBF9D
:101630000FBECDBFCF91DF911F910F91FF90EF9023
:10164000DF90CF90BF90AF909F908F9008958F9232
:101650009F92AF92BF92CF92DF92EF92FF920F9341
:101660001F93DF93CF93CDB7DEB72E970FB6F894C5
:10167000DEBF0FBECDBF19821A821B821C828091F1
:10168000A8019091A9018E010B5F1F4FB8014AE09C
:1016900050E00E94B818F80101900020E9F7319756
:1016A000FE2EF01A80E0CF2CDD24C7FCD094AAE0F7
:1016B0008A2E912C8C0E9D1E58010BC0F501E00F57
:1016C000F11F80810E94DC05080D191DF80180833F
:1016D0008E2D082F10E0E82EE3940C151D0574F3F1
:1016E00080939F0385E166E0AE014F5F5F4F24E08A
:1016F0000E94BE0989E18F1966E0A4012F2D0E9486
:10170000BE098091A8019091A9011816190664F4E8
:1017100085E060E00E94A20286E062EC0E94A202E4
:1017200087E06CE80E94A2028091A8019091A90133
:1017300097FF0CC085E060E00E94A20286E062ECA8
:101740000E94A20287E06DE80E94A2028091A80197
:101750009091A901892B61F485E060E00E94A202CA
:1017600086E062EC0E94A20287E060E00E94A20292
:101770002E960FB6F894DEBF0FBECDBFCF91DF918E
:101780001F910F91FF90EF90DF90CF90BF90AF909F
:101790009F908F9008958F929F92AF92BF92CF9219
:1017A000DF92EF92FF920F931F93DF93CF93CDB70A
:1017B000DEB72B970FB6F894DEBF0FBECDBFDE01AC
:1017C0001196EEE3F1E083E001900D928150E1F794
:1017D0008E010C5F1F4F8091140390911503B80187
:1017E0004AE050E00E94B818F80101900020E9F7A3
:1017F0003197FE2EF01A80E0CF2CDD24C7FCD09468
:10180000B8E08B2E912C8C0E9D1E58010BC0F5015B
:10181000E00FF11F80810E94DC05080D191DF80101
:1018200080838E2D082F10E0E82EE3940C151D0503
:1018300074F380939F038DE06EE0AE014F5F5F4FC6
:1018400023E00E94BE0980E18F196EE0A4012F2DD4
:101850000E94BE092B960FB6F894DEBF0FBECDBF17
:10186000CF91DF911F910F91FF90EF90DF90CF907C
:10187000BF90AF909F908F9008958F929F92AF925C
:10188000BF92DF92EF92FF920F931F93DF93CF935C
:10189000CDB7DEB728970FB6F894DEBF0FBECDBF29
:1018A00019828AE08A8380919A0190919B018E012E
:1018B0000D5F1F4FB8014AE050E00E94B818F801D0
:1018C00001900020E9F73197E01B80E0EE2EFF2425
:1018D000E7FCF094480106E0A02EB12CAC0EBD1E32
:1018E0000BC0F401E00FF11F80810E94DC050A0D9E
:1018F0001B1DF80180838D2D082F10E0D82ED39466
:101900000E151F0574F380939F0380919A019091A7
:101910009B018E010A5F1F4F0A977CF460910301BF
:1019200081E0AE014F5F5F4F21E00E94BE096091F0
:10193000030182E0A80121E005C06091030181E07C
:10194000A80122E00E94BE0980919C0190919D0116
:101950008E010D5F1F4FB8014AE050E00E94B81899
:10196000F80101900020E9F73197E01B80E0EE2EAE
:10197000FF24E7FCF094480116E0A12EB12CAC0E38
:10198000BD1E0BC0F401E00FF11F80810E94DC0539
:101990000A0D1B1DF80180838D2D082F10E0D82E15
:1019A000D3940E151F0574F380939F0380919C01BF
:1019B00090919D018E010A5F1F4F0A977CF4609100
:1019C000030184E0AE014E5F5F4F21E00E94BE093B
:1019D0006091030185E0A80121E005C06091030149
:1019E00084E0A80122E00E94BE0928960FB6F89470
:1019F000DEBF0FBECDBFCF91DF911F910F91FF9042
:101A0000EF90DF90BF90AF909F908F9008950F93CD
:101A10001F93DF93CF93CDB7DEB72A970FB6F89415
:101A2000DEBF0FBECDBF8E010F5F1F4FB8014AE072
:101A300050E00E94B818F80101900020E9F73197B2
:101A4000E01B20E0FF27E7FDF095322F3F5F822F5C
:101A500090E08E179F0714F4232FF7CF20939F0356
:101A60002A960FB6F894DEBF0FBECDBFCF91DF919F
:101A70001F910F910895AF92BF92CF92DF92EF9294
:101A8000FF920F931F93DF93CF93CDB7DEB76E977F
:101A90000FB6F894DEBF0FBECDBFB82EA62ED42E43
:101AA000A42FB52FFD0101900020E9F73197CE2E2C
:101AB000C41A7E010894E11CF11C242F352FC901A2
:101AC0008C0108C0F80181918F010E94DC05F701AB
:101AD00081937F01802F8D198C15A0F38B2D6A2D9A
:101AE000AE014F5F5F4F2C2D0E94BE096E960FB660
:101AF000F894DEBF0FBECDBFCF91DF911F910F9144
:101B0000FF90EF90DF90CF90BF90AF9008958091BD
:101B10009201813069F4609106018091D70187FDBF
:101B20008F5F85958195825F48ED51E00E943B0D66
:101B30000895EF92FF920F931F93DF93CF93CDB74A
:101B4000DEB764970FB6F894DEBF0FBECDBFF82E98
:101B5000E62ECA018E010F5F1F4FB8014AE050E028
:101B60000E94B8188F2D6E2DA8010E943B0D64961F
:101B70000FB6F894DEBF0FBECDBFCF91DF911F919E
:101B80000F91FF90EF900895BF92CF92DF92EF9266
:101B9000FF920F931F93DF93CF93CDB7DEB7649778
:101BA0000FB6F894DEBF0FBECDBFC82EB62EFA0119
:101BB0007E010894E11CF11C04C0AE0DBF1D9C9376
:101BC00031968E2F841B9491A82FB0E09923A9F70A
:101BD000AE0DBF1D1C92F70101900020E9F731976F
:101BE000DE2EDE18870107C0F80180810E94DC0527
:101BF000F80181938F01802F8E198D15A8F38C2DFC
:101C00006B2DAE014F5F5F4F2D2D0E94BE09649674
:101C10000FB6F894DEBF0FBECDBFCF91DF911F91FD
:101C20000F91FF90EF90DF90CF90BF9008951F939A
:101C3000CF93DF93EC01A3E0B0E047C0FD01E4598E
:101C4000FD4F8081FD01E359FD4F2081422F50E07F
:101C50004D535040FD01E259FD4F7081FD01E159A6
:101C6000FD4F10819A01F4E035952795FA95E1F73B
:101C700090E0CD97880F991F880F991F282B392B3B
:101C80002883613029F1E72FF0E0FD9734E0440F1D
:101C9000551F3A95E1F75070CF0195958795959529
:101CA0008795482B592B4983623091F014966350E5
:101CB00086E0EE0FFF1F8A95E1F7F070812F90E02C
:101CC000CD97E82BF92BEA832396662309F0B6CF4C
:101CD000DF91CF911F91089580916E028635B1F406
:101CE00080916D0281568093B4018091B40184305B
:101CF00018F084E08093B40184E493E06AE043E068
:101D00002AE00E94170E81E08093B50110928F01A6
:101D100008951F931091B401123009F48AC0143051
:101D200009F4E3C0113009F0A7C180916E0281353A
:101D300081F480E893E06BE143E02DE20E94170E0E
:101D40008091800390E09093B7018093B601109347
:101D5000BA0180916E02843409F08EC182E093E072
:101D600061E443E021E40E94170E809118039091F2
:101D70001903843B910554F480919401813031F42E
:101D800010929401F8940E94501078948091180356
:101D900090911903843B91057CF0809194018823F4
:101DA00059F481E080939401F89480919101882303
:101DB00011F40E94401078948091040390910503DF
:101DC00066E170E00E9409196E5F7F4F70934502D3
:101DD00060934402809106039091070366E170E0EE
:101DE0000E9409196A5F7F4F709343026093420219
:101DF00080910E0390910F036EE170E00E9409192B
:101E000070934702609346028091160380934A02C2
:101E10008091290290912A0290934902809348026E
:101E2000809114039091150390934D0280934C027E
:101E300023C180916E028F34A9F0813509F01CC155
:101E400080E893E06BE143E02DE20E94170E809161
:101E5000800390E09093B7018093B60181E0809376
:101E6000BA010AC18CEE91E060E543E02DE20E94E8
:101E7000170E80913402992787FD909502969093D2
:101E800045028093440280913502992787FD909501
:101E9000069690934302809342028091270290918C
:101EA00028026EE170E00E94091970934702609366
:101EB000460280912D0280934A02809129029091DE
:101EC0002A029093490280934802809132029091B5
:101ED000330290934D0280934C02809126028093AE
:101EE0004E0281E08093B901C7C080916E028434B4
:101EF00009F05EC082E093E061E443E021E40E94E7
:101F0000170E8091180390911903843B910554F4A6
:101F100080919401813031F410929401F8940E94E0
:101F2000501078948091180390911903843B910587
:101F30007CF080919401882359F481E0809394018E
:101F4000F89480919101882311F40E9440107894B4
:101F5000809104039091050366E170E00E940919E5
:101F60006E5F7F4F70934502609344028091060339
:101F70009091070366E170E00E9409196A5F7F4F44
:101F8000709343026093420280910E0390910F037D
:101F90006EE170E00E940919709347026093460257
:101FA000809114039091150390934D0280934C02FD
:101FB00080916E028C3481F481E090E09093B701BF
:101FC0008093B60181E08093BA0182E893E069E1F1
:101FD00043E02DE20E94170E80916E028D3481F451
:101FE00082E090E09093B7018093B60181E0809306
:101FF000BA0182E893E069E143E02DE20E94170E06
:1020000080916E028E3481F483E090E09093B7016A
:102010008093B60181E08093BA0182E893E069E1A0
:1020200043E02DE20E94170E80916E028F3481F4FE
:1020300084E090E09093B7018093B60181E08093B3
:10204000BA0182E893E069E143E02DE20E94170EB5
:1020500080916E02803581F485E090E09093B70125
:102060008093B60181E08093BA0182E893E069E150
:1020700043E02DE20E94170E10928F011F910895E8
:1020800082E289B910BC80B91CBE909A28E92AB9AD
:1020900096E890BD82EC8BB921B99CBF82B90895B6
:1020A00082E289B910BC80B91CBE88E98AB926E8E9
:1020B00020BD92EC9BB980E981B92CBF92B90895FB
:1020C000DF93CF93CDB7DEB72C970FB6F894DEBF72
:1020D0000FBECDBF83E2898383E68A8385E78B8346
:1020E0008DE38C838D838E838F83DE011196FD01BA
:1020F00020E030E0AE01485F5F4F8191280F311D35
:10210000E417F507D1F7C9019F7046E095958795CB
:102110004A95E1F7835C88872F733070822F835C48
:1021200089878DE08A879E01255F3F4F8C91159BA3
:10213000FECF83B91196A217B307C1F72C960FB63D
:10214000F894DEBF0FBECDBFCF91DF910895DF932E
:10215000CF93CDB7DEB72C970FB6F894DEBF0FBE86
:10216000CDBF8BE189838A8385E58B838AEA8C8363
:102170001D82FE0131969E012A5F3F4F8081159B93
:10218000FECF83B93196E217F307C1F72C960FB64D
:10219000F894DEBF0FBECDBFCF91DF910895DF93DE
:1021A000CF93CDB7DEB72A970FB6F894DEBF0FBE38
:1021B000CDBF93E299838A836B83842F869586951E
:1021C000835C8C8350E04370507064E0440F551F73
:1021D0006A95E1F7435C4D838DE38E838F83DE0147
:1021E0001196FD0120E030E0AE01485F5F4F819124
:1021F000280F311DE417F507D1F7C9019F7056E08C
:10220000959587955A95E1F7835C88872F73307091
:10221000822F835C89878DE08A879E01255F3F4FEF
:102220008C91159BFECF83B91196A217B307C1F706
:102230002A960FB6F894DEBF0FBECDBFCF91DF91C7
:1022400008955D9BFECF8DE68CB95D9BFECF8FE63A
:102250008CB95D9BFECF89E68CB95D9BFECF8EE687
:102260008CB95D9BFECF8DE08CB95D9BFECF8EE37C
:102270008CB90895159BFECF83B908955D9BFECF61
:102280008CB90895662359F020E0FC01E20FF11D9E
:10229000E0815D9BFECFECB92F5F6217B0F7089528
:1022A0005D9BFECF8EE38CB908951F920F920FB6FF
:1022B0000F9211242F933F938F939F93AF93BF93CC
:1022C000EF93FF932CB12093A00385B398E0892767
:1022D00085BB5D9BFECF2CB92D3059F080917F03DB
:1022E000E82FF0E0E75AFC4F20838F5F80937F0355
:1022F00059C0E0917F03F0E0E75AFC4F2083109231
:10230000B1011092B2011092B30120E030E090E0F0
:102310003FC02130B9F0213018F02230C1F524C07F
:10232000A32FB0E0A75ABC4F8C91803211F421E06A
:1023300023C0E92FF0E08C91E958FC4F8083909303
:10234000B10124C0A32FB0E0A75ABC4F8C918032BA
:1023500011F422E011C0E92FF0E08C91E15AFD4F19
:1023600080839093B20112C0A32FB0E0A75ABC4F54
:102370008C91803219F423E090E009C0E92FF0E05D
:102380008C91E05BFD4F80839093B3019F5F3F5F33
:1023900080917F03831708F0BCCF81E08093B00168
:1023A00010927F03FF91EF91BF91AF919F918F9119
:1023B0003F912F910F900FBE0F901F9018951F9275
:1023C0000F920FB60F9211248F939F93EF93FF9369
:1023D00093B19093A1039D3081F48091C401813029
:1023E00061F4AB981092C40180938F01E0914F0388
:1023F000F0E0E459FD4F90832DC08091C401882303
:1024000019F0813039F514C0933241F480918F0175
:10241000882321F481E08093C401AB9A10924F038A
:1024200080914F03E82FF0E0E459FD4F90830CC0FA
:10243000E0914F03F0E0E459FD4F908380914F030A
:10244000853930F480914F038F5F80934F0302C032
:102450001092C401FF91EF919F918F910F900FBE49
:102460000F901F90189585B392E0892785BB08953A
:1024700090919701913019F485B3892785BB089510
:102480001F920F920FB60F9211242F933F935F93D9
:102490006F937F938F939F93AF93BF938091C60168
:1024A0009091C701892B81F484B595B59093CD01A6
:1024B0008093CC018EB58F7B8EBD81E090E09093B0
:1024C000C7018093C6013AC084B595B59093CB01FE
:1024D0008093CA012EB520642EBD2091CC0130918D
:1024E000CD011092C7011092C601821B930B865634
:1024F00098406CE271E00E94F5187093C9016093F6
:10250000C8016730710534F086E090E09093C9010E
:102510008093C8012091C8013091C90180910201C6
:10252000992787FD90952817390741F02630310506
:102530002CF42093020181E080939E01BF91AF9122
:102540009F918F917F916F915F913F912F910F900C
:102550000FBE0F901F9018958091460290914702F0
:102560009093A1018093A0018091A0019091A1017D
:102570002091A2013091A301821B930B9093A5019E
:102580008093A4018091A0019091A1019093A30157
:102590008093A2014091AC015091AD018091A401C2
:1025A0009091A501E3E0880F991FEA95E1F79A0160
:1025B00073E0220F331F7A95E1F7241B350B820F4E
:1025C000931F68E070E00E9409197093AD01609359
:1025D000AC012091AE013091AF014091AC0150911E
:1025E000AD01C90163E0880F991F6A95E1F7821B6D
:1025F000930B840F951F68E070E00E940919709397
:10260000AF016093AE018091AE019091AF019093C4
:10261000A9018093A8010E94270B08958F929F9291
:10262000BF92CF92DF92EF92FF920F931F93DF93AF
:10263000CF93CDB7DEB72B970FB6F894DEBF0FBEA2
:10264000CDBFDE011196E0E5F1E083E001900D924F
:102650008150E1F780914E028E010C5F1F4F90E098
:10266000B8014AE050E00E94B818F801019000203B
:10267000E9F73197BE2EB01AEE24FF24CB2CDD24CF
:10268000C7FCD09488E0882E912C8C0E9D1E0DC026
:10269000F801EE0DFF1D80810E94DC05F401EE0DB6
:1026A000FF1D80830894E11CF11CEC14FD0484F3ED
:1026B00088E161E0AE014F5F5F4F23E00E94BE09F9
:1026C0008BE18B1961E0A4012B2D0E94BE092B9692
:1026D0000FB6F894DEBF0FBECDBFCF91DF911F9133
:1026E0000F91FF90EF90DF90CF90BF909F908F90D1
:1026F00008958AE161E04EE451E022E00E94BE09C3
:10270000089583E66FE644E60E94CF10F89428E02F
:1027100088E190E00FB6F894A89581BD0FBE21BD69
:10272000FFCF1F939D998AC18091CE018F5F8093C7
:10273000CE0111E01093D0018091CE01853009F0D7
:1027400081C18091D201882309F08CC01093D201FD
:102750001092D30184E064E00E94A20283E061E071
:1027600048ED51E00E943B0D83E063E042E152E01E
:102770000E94C40D84E068E00E94A20283E065E04C
:102780004BE152E00E94C40D80910001813029F498
:1027900084E165E047E452E004C084E165E04AE496
:1027A00052E00E94C40D84E060E00E94A20283E037
:1027B00066E04FE152E00E94C40D809191018130AA
:1027C00029F484E166E047E452E004C084E166E075
:1027D0004AE452E00E94C40D83E067E045E252E023
:1027E0000E94C40D80919201813029F484E167E058
:1027F00047E452E004C084E167E04AE452E00E940A
:10280000C40D83E068E04DE252E00E94C40D809167
:102810009F01813029F484E168E047E452E004C07C
:1028200084E168E04AE452E00E94C40D83E069E07C
:1028300048E352E00E94C40D80919301813029F455
:1028400084E169E047E452E004C084E169E04AE4DD
:1028500052E00E94C40D83E06BE042E452E00E942B
:10286000C40DEEC08091D301882349F584E068E06F
:102870000E94A20280910001882339F41093000184
:1028800084E165E047E452E006C01092000184E173
:1028900065E04AE452E00E94C40D20910001E199F4
:1028A000FECF81E090E09FBB8EBB2DBB0FB6F894AE
:1028B000E29AE19A0FBE84E060E00E94A2021091C9
:1028C000D301113049F584E068E00E94A2028091B2
:1028D0009101882339F41093910184E166E047E483
:1028E00052E006C01092910184E166E04AE452E0B1
:1028F0000E94C40D20919101E199FECF80E090E00B
:102900009FBB8EBB2DBB0FB6F894E29AE19A0FBE27
:1029100084E060E00E94A2028091D301823051F5F0
:1029200084E068E00E94A20280919201882341F431
:1029300081E08093920184E167E047E452E006C0C1
:102940001092920184E167E04AE452E00E94C40DD3
:1029500020919201E199FECF82E090E09FBB8EBB77
:102960002DBB0FB6F894E29AE19A0FBE84E060E0C6
:102970000E94A2028091D301833051F584E068E087
:102980000E94A20280919F01882341F481E08093FC
:102990009F0184E168E047E452E006C010929F0185
:1029A00084E168E04AE452E00E94C40D20919F0156
:1029B000E199FECF87E190E09FBB8EBB2DBB0FB6A8
:1029C000F894E29AE19A0FBE84E060E00E94A202CD
:1029D0008091D301843049F568E00E94A202809181
:1029E0009301882341F481E08093930184E169E0BD
:1029F00047E452E006C01092930184E169E04AE4A2
:102A000052E00E94C40D20919301E199FECF8BE129
:102A100090E09FBB8EBB2DBB0FB6F894E29AE19A73
:102A20000FBE84E060E00E94A2028091D301853055
:102A300049F41092D2010E94811304C01092CE0179
:102A40001092D0019C9913C19091D201913009F05C
:102A500014C19093D1018091CF018F5F8093CF01FA
:102A60002091CF01253009F008C11092CF0180914B
:102A7000D301823009F469C0833030F4882371F0C7
:102A8000813009F0FAC035C0843009F4AAC084301E
:102A900008F486C0853009F0F0C0C3C09093D3011C
:102AA00083E065E04BE152E00E94C40D809100019B
:102AB000813029F484E165E047E452E004C084E118
:102AC00065E04AE452E00E94C40D84E068E00E94A0
:102AD000A20283E066E04FE152E00E94C40D8091C3
:102AE0009101813019F484E166E0B3C084E166E0CD
:102AF000B5C082E08093D30183E066E04FE152E00D
:102B00000E94C40D80919101813029F484E166E036
:102B100047E452E004C084E166E04AE452E00E94E7
:102B2000C40D84E068E00E94A20283E067E045E211
:102B300052E00E94C40D80919201813019F484E129
:102B400067E087C084E167E089C083E08093D301B8
:102B500067E045E252E00E94C40D8091920181300D
:102B600029F484E167E047E452E004C084E167E0CF
:102B70004AE452E00E94C40D84E068E00E94A20290
:102B800083E068E04DE252E00E94C40D80919F0115
:102B9000813019F484E168E05CC084E168E05EC0E3
:102BA00084E08093D30183E068E04DE252E00E942C
:102BB000C40D80919F01813029F484E168E047E4ED
:102BC00052E004C084E168E04AE452E00E94C40D8F
:102BD00084E068E00E94A20283E069E048E352E0FA
:102BE0003FC02093D30183E069E048E352E00E94B4
:102BF000C40D80919301813029F484E169E047E4B8
:102C000052E004C084E169E04AE452E00E94C40D4D
:102C100084E068E00E94A20283E06BE042E452E0BC
:102C20001FC01092D30183E06BE042E452E00E94A7
:102C3000C40D84E068E00E94A20283E065E04BE1FD
:102C400052E00E94C40D80910001813029F484E19A
:102C500065E047E452E004C084E165E04AE452E004
:102C60000E94C40D84E060E00E94A20206C010929F
:102C7000CF018091D0018091D1011F9108958130C1
:102C800061F4E199FECF80E090E09FBB8EBB6DBB0D
:102C90000FB6F894E29AE19A0FBE0895DF93CF93AE
:102CA000CDB7DEB764970FB6F894DEBF0FBECDBFC9
:102CB00020E0BE016F5F7F4F422F50E0E199FECFD1
:102CC000822F90E08D5F9F4F9FBB8EBBE09A8DB3AC
:102CD000FB01E40FF51F80838823A9F08F3F11F4D7
:102CE000108211C02F5FE8CFFD01E852FE4FA40F04
:102CF000B51F8C91808311829F5FA92FB0E0A2172E
:102D0000B30794F312C0DE011196FD01019000207B
:102D1000E9F73197EA1BFB0BE093D70190E02E2FE8
:102D2000332727FD3095AD01E8CF64960FB6F894B0
:102D3000DEBF0FBECDBFCF91DF910895DF93CF935C
:102D4000CDB7DEB760970FB6F894DEBF0FBECDBF2C
:102D500080914C0290914D0290936B0280936A0295
:102D600080916A0290916B026FE070E00E94F5180A
:102D7000DE011596AD016A1B9E01205F3F4FE62FD5
:102D8000EA0FF0E0E35BFD4FE491ED93A217B30788
:102D9000B1F76091070119821A821B821C8289E0B7
:102DA0002BE00E94BE09609108018EE0AE014F5FEA
:102DB0005F4F24E00E94BE096091080140916A02C1
:102DC00050916B028FE00E94990D60960FB6F894B7
:102DD000DEBF0FBECDBFCF91DF910895DF93CF93BC
:102DE000CDB7DEB7E4970FB6F894DEBF0FBECDBF08
:102DF000DE011796E3E5F1E087E001900D92815046
:102E0000E1F7DE011E96EAE5F1E089E001900D921E
:102E10008150E1F7DE015796E3E6F1E08EE00190A4
:102E20000D928150E1F7DE011196E1E7F1E086E0D5
:102E300001900D928150E1F7DE019596E7E7F1E010
:102E400080E101900D928150E1F7509177036091FC
:102E500078034091790380917A0320E030E0803755
:102E600011F421E030E080E090E04C3611F481E094
:102E700090E02823392380E0583609F481E090E07F
:102E8000653609F491E0892390E028233923232B28
:102E900079F0CE01079666E00E944211CE010E96AF
:102EA00068E00E944211CE0147966DE00E944211F7
:102EB00050917703609178034091790380917A0370
:102EC00020E030E0873711F421E030E080E090E04E
:102ED0004F3611F481E090E02823392380E0533706
:102EE00009F481E090E0683609F491E0892390E0EC
:102EF00028233923232B19F180915F0290916002DE
:102F0000893481F4943471F4CE01019665E00E9415
:102F1000421188ED91E06091D7010E9442118DE04D
:102F20000E943E1180915F0290916002863739F4D1
:102F3000953629F4CE01859668E00E944211809171
:102F40007703209178034091790390E0833709F467
:102F500091E080E0253609F481E09823892F90E004
:102F600020E030E0443711F421E030E08223932365
:102F7000892B09F440C080915F02909160028934EE
:102F800009F039C0943409F036C020E01CC0A22FEB
:102F9000B0E0FD01E05BFD4FE081E199FECF822FC3
:102FA00090E08D5F9F4F9FBB8EBBEDBB0FB6F8943B
:102FB000E29AE19A0FBEFD01E05BFD4F8081A852CD
:102FC000BE4F8C932F5F8091B301281700F3E199D6
:102FD000FECFE22FF0E0CF018D5F9F4F9FBB8EBBF6
:102FE0001DBA0FB6F894E29AE19A0FBEE852FE4F6E
:102FF00010822093D701509177036091780340911C
:10300000790380917A0320E030E0853611F421E0E5
:1030100030E080E090E0433711F481E090E0282335
:10302000392380E0523709F481E090E0653609F4F5
:1030300091E0892390E028233923232B11F00E946B
:1030400081130E945011E4960FB6F894DEBF0FBEB4
:10305000CDBFCF91DF91089583ED8DB90895813073
:1030600031F4613011F492980895929A0895823063
:1030700029F4613011F494980895949A08951F9258
:103080000F920FB60F9211242F933F934F935F939C
:103090006F937F938F939F93AF93BF93EF93FF9320
:1030A0008091D501882369F08091D50190E0019746
:1030B000E0918801F0918901E80FF91F8FB18083B9
:1030C00003C08FB18093A9032091D501809187011E
:1030D00030E0992787FD90958217930754F087E099
:1030E0008093A8031092A6038091D5018093A70333
:1030F00009C081E060E00E942F181092D40181E0A5
:103100008093D6018091D5018F5F8093D501FF9187
:10311000EF91BF91AF919F918F917F916F915F914F
:103120004F913F912F910F900FBE0F901F901895C8
:103130001F93182F8091D401882311F081E016C0CD
:10314000812F61E00E942F181093D401113069F48F
:1031500086E0809387011092D50183E08093A803D5
:103160001092A6038AEA8093A70380E01F91089536
:10317000FB019F01E8944230C4F04532B4F44A3078
:1031800029F497FB1EF4909581959F4F642F772724
:103190000E94F518805D8A330CF0895D8193CB0124
:1031A0000097A1F716F45DE251931082C9010C94C7
:1031B000D918DC01FC01672F71917723E1F7329771
:1031C00004C07C916D9370836291AE17BF07C8F302
:1031D0000895991B79E004C0991F961708F0961B73
:1031E000881F7A95C9F780950895AA1BBB1B51E1EA
:1031F00007C0AA1FBB1FA617B70710F0A61BB70B67
:10320000881F991F5A95A9F780959095BC01CD010B
:10321000089597FB092E07260AD077FD04D0E5DF35
:1032200006D000201AF4709561957F4F0895F6F747
:0C323000909581959F4F0895F894FFCF72
:10323C000101030E0786010E0C5C00000A0000441D
:10324C0000002300230054646653636552620051EE
:10325C006100506000506000516100526200536385
:10326C00655464666768696A6B6B6A6968670000B5
:10327C000053536353530203EC0180030D0A0A1DE0
:10328C0000000068656C70200D0073686F77204932
:10329C00440D0073686F772076657273696F6E0DDD
:1032AC00004944203D2000302E392E312E302E6125
:0A32BC002E626574610D00085203D4
:00000001FF
